:020000040801F1
:10000000A0790120A10101082B1401080D1301089A
:1000100029140108AD020108691901080000000057
:100020000000000000000000000000002F14010884
:10003000AF020108000000002D140108311401086E
:10004000BB010108BB010108BB010108BB0101089C
:10005000BB010108BB010108BB010108BB0101088C
:10006000BB010108BB010108BB010108BB0101087C
:10007000BB010108BB010108BB010108BB0101086C
:10008000BB010108BB010108BB010108BB0101085C
:10009000BB010108BB010108BB010108BB0101084C
:1000A000BB010108BB010108BB010108BB0101083C
:1000B000BB010108BB010108BB010108BB0101082C
:1000C000BB010108BB010108BB010108BB0101081C
:1000D000BB010108511901085D190108BB010108A4
:1000E000BB010108BB010108BB010108BB010108FC
:1000F000BB010108BB010108BB010108BB010108EC
:10010000BB010108BB010108BB010108BB010108DB
:100110000D150108BB010108BB010108BB01010865
:10012000BB010108BB010108BB010108BB010108BB
:10013000BB010108BB010108BB010108BB010108AB
:10014000BB010108BB010108BB010108BB0101089B
:10015000BB010108BB010108BB010108BB0101088B
:10016000BB010108BB010108BB010108BB0101087B
:10017000BB010108BB010108BB0101080000000030
:10018000BB010108BB010108DFF810D000F07CF8CA
:1001900000480047C91C0108AFF30080A079012086
:1001A0000648804706480047FEE7FEE7FEE7FEE711
:1001B000FEE7FEE7FEE7FEE7FEE7FEE7B51401080F
:1001C000890101082DE9F05F0546002092469B4613
:1001D00088460646814640241BE02846414647465D
:1001E000224600F041F853465A46C01A914110D3B6
:1001F00011461846224600F028F82D1A67EB010830
:100200004F4622460120002100F01FF817EB00099D
:100210004E41201EA4F10104DFDC484631462A4647
:100220004346BDE8F09FD2B201E000F8012B491E21
:10023000FBD270470022F6E710B513460A46044683
:100240001946FFF7F0FF204610BD202A04DB203AB4
:1002500000FA02F1002070479140C2F1200320FA19
:1002600003F3194390407047202A04DB203A21FA17
:1002700002F00021704721FA02F3D040C2F12002BF
:100280009140084319467047064C074D06E0E06868
:1002900040F0010394E8070098471034AC42F6D3CD
:1002A000FFF776FF441E0108641E0108FEE7704751
:1002B00070470000002229B101291AD002291BD061
:1002C0004FF440720E490B6823F440730B600B68C7
:1002D00013430B600A6822F0F8020A600A680223DE
:1002E00003EBC00002430A60086840F480300860F5
:1002F00070474FF48072E5E74FF40072E2E70000C8
:10030000103C02401348016889050FD5016821F4AB
:1003100000710160016841F400610160016821F42D
:1003200000610160016841F40071016001684905E4
:100330000FD5016821F480610160016841F48051AA
:100340000160016821F480510160016841F480611D
:1003500001607047003C024008490A6822F440727C
:100360000A600A6842F004020A600A684FF48033A7
:1003700043EA002002430A6070470000103C02403C
:10038000064A136823F440731360136813601368FC
:1003900043F001031360017070470000103C0240FD
:1003A000084910B50C6824F440740C600C6844F4DF
:1003B00040740C600C6844F001040C6002604360FF
:1003C00010BD0000103C0240074A136823F440733C
:1003D0001360136843F480731360136843F00103E0
:1003E0001360018070470000103C0240074A136808
:1003F00023F440731360136843F4007313601368AD
:1004000043F001031360016070470000103C02409C
:1004100017490868C206174805D5C26942F010029C
:10042000C26110220A600A68920605D5C26942F0CC
:100430000802C26120220A600A68520605D5C26914
:1004400042F00402C26140220A600A68120605D521
:10045000C26942F00202C26180220A600A68920701
:1004600005D5C26942F02002C261022008607047CF
:100470000C3C02408039012070B51149044600202F
:10048000C86100F0BBF906460E4D09E0601C07D0BC
:1004900024B100F0B3F9801BA04201D9032070BD44
:1004A0002868C003F2D42868C00701D00120286062
:1004B000286810F0F200F2D0FFF7AAFF012070BD0B
:1004C000803901200C3C024090F83510022903D0FD
:1004D0008021416501207047052180F835100068B2
:1004E000016821F001010160002070472DE9F0470B
:1004F000044622480F46017E01290AD00121804688
:1005000001764CF250394846FFF7B6FF020003D09F
:100510002FE00220BDE8F0874FF0FF303860206800
:10052000174D012801D0A6681CE0207C6168FFF708
:1005300013FF4846FFF7A0FF0246286820F004009A
:10054000286014E0217C3046FFF7B4FE4846FFF7F0
:1005500093FF0200286820F0FA00286001D03E6076
:1005600005E0761CD4E902100844B042EAD8FFF74F
:10057000C9FE002188F818101046CBE78039012009
:10058000103C02400348016841F000410160002036
:1005900070470000103C02402DE9F0471B4E054615
:1005A0001446307E1F468946012808D00120307647
:1005B0004CF250384046FFF75FFF18B114E00220BC
:1005C000BDE8F0879DB1012D16D0022D19D022462D
:1005D0003B464846FFF7E4FE4046FFF74DFF0C4917
:1005E0000A6822F001020A6000213176E8E7E1B2F0
:1005F0004846FFF7C5FEEFE7A1B24846FFF7E4FE25
:10060000EAE721464846FFF7F1FEE5E78039012099
:10061000103C0240074900200A68002A09DA054A0E
:10062000054B0C3A1360054B13600968002900DA8A
:1006300001207047103C024023016745AB89EFCD94
:100640002DE9F84FDFF87CB100224FF001084FF0A0
:10065000030A4FF00F090BF1040E00BF0B6808FAF4
:1006600002F42340A3426ED14D68022D01D0122D19
:100670000ED1D50800EB850CDCF820505607F70E9C
:1006800009FA07F6B5430E69BE402E43CCF8206048
:10069000066855000F790AFA05FC07F0030726EAF9
:1006A0000C06AF40374307604E68012E05D0022E7E
:1006B00003D0112E01D0122E0ED18668CF6826EA03
:1006C0000C06AF40374387604668A6430C79C4F3F5
:1006D0000014944034434460C6688C6826EA0C06D3
:1006E000AC403443C4604C68E40065D5364C2568A2
:1006F00045F480452560246822F0030504F4804415
:100700000094324C2E19D6F8084895072F0F09FA95
:1007100007F5AC432E4DA84201D1002524E02D4D14
:10072000A84201D101251FE02B4DA84201D102258D
:100730001AE02A4DA84201D1032515E0284DA84210
:1007400002D1042510E037E0264DA84201D105254D
:100750000AE0254DA84201D1062505E0234DA84217
:1007600001D1072500E00825BD402543C6F80858FB
:10077000DBF800405D464E689C43F60300D51C4301
:100780002C60DEF8004075464E689C43B60300D5E9
:100790001C432C600B4D08352C684E689C43F602B8
:1007A00000D51C432C60074D0C352C684E689C43CB
:1007B000B60200D51C432C60521C102AFFF44EAF29
:1007C000BDE8F88F003C0140443802400030014051
:1007D000000002400004024000080240000C0240F9
:1007E000001002400014024000180240001C0240A9
:1007F0000AB1816170470904FBE700000148806885
:10080000704700001C0000200248816802781144F3
:10081000816070471C0000200B4810B5016841F44E
:1008200000710160016841F480610160016841F478
:1008300080710160032000F06FF8002000F006F8DE
:1008400000F024F8002010BD003C024070B50D4DB2
:1008500004464FF47A712878B1FBF0F00A49096830
:10086000B1FBF0F000F0E2FA48B9102C07D20022F8
:100870002146501E00F030F800206C6070BD012051
:1008800070BD00001C000020280000200A4808B5A8
:10089000016841F480410160006800F480400090EC
:1008A0000548001F016841F080510160006800F0B8
:1008B0008050009008BD000044380240002809DB49
:1008C00000F01F02012191404009800000F1E0206A
:1008D000C0F8001170470000F0B40E4B1B680C46C6
:1008E000C3F30223C3F10705042D00D90425191D04
:1008F000072901D2002300E0DB1E012606FA05F1DC
:10090000491E214099409E40761E16403143F0BC5E
:1009100001F04EB80CED00E0064900F0070208684F
:100920004FF6FF03184040EA0220034A10430860D4
:10093000704700000CED00E00000FA052DE9F047DB
:100940000E46050065D0DFF81481D8F80000F7B234
:1009500000F00F00B04207D288F80070D8F800000D
:1009600000F00F00B04254D128683D4C810712D5E9
:10097000400703D5206840F4E05020602878000745
:1009800003D5206840F4604020602068A96820F00A
:10099000F000084320602878C0072DD030496868EF
:1009A0000839012812D0022813D0032811D0096871
:1009B000890700292DDA216821F003010143216014
:1009C000FFF71CFF814641F2883A0EE0096889036F
:1009D000EFE709688901ECE7FFF710FFA0EB0901D9
:1009E000514502D90320BDE8F0872068696800F00E
:1009F0000C00B0EB810FEFD1D8F80010404601F0A9
:100A00000F01B14207D90770006800F00F00B04233
:100A100001D00120E7E72878400705D52068E9687C
:100A200020F4E050084320602878000706D52068AD
:100A3000296920F4604040EAC100206000F036F8E7
:100A40002168084AC1F30311515CC8400649086097
:100A50000020FFF7FBFE0020C5E70000003C02403D
:100A6000083802402C1E01082800002004480549CF
:100A700000680968044AC1F38221515CC84070478C
:100A800028000020083802403C1E0108044805499F
:100A900000680968044AC1F34231515CC84070479C
:100AA00028000020083802403C1E0108154810B5F7
:100AB000006810F00C02144813D01449042A0FD017
:100AC000082A0ED10F4C241F2268236802F03F022F
:100AD0005B0207D52068C0F38810A0FB010106E087
:100AE000084610BD2168C1F38811A1FB0001002355
:100AF000FFF768FB2168C1F30141491C4900B0FBC5
:100B0000F1F010BD083802400024F40040787D0167
:100B10002DE9F84F050076D02878DFF8F8B2BE4C02
:100B2000C00749D0DBF800105846C1F38101012904
:100B300008D00068C0F3810002280AD1201D006897
:100B4000400206D52068800336D568680028E2D0C8
:100B500032E06868B0F5803F10D0B0F5A02F206873
:100B600010D020F480302060206820F480202060A5
:100B70006868A0B1FFF742FE06460CE0206840F42A
:100B80008030F4E740F480202060F7E7FFF736FE7E
:100B9000801B642873D820688003F7D50CE0FFF72A
:100BA0002DFE064605E000BFFFF728FE801B6428E7
:100BB000F0D820688003F7D42878DFF860828007B7
:100BC0004FF000093ED5DBF80010584611F00C0F2D
:100BD00009D00068C0F3810002280BD18D48001FA6
:100BE0000068400206D42068800715D5E86801280F
:100BF00009D111E0E868B8B10120C8F80000FFF79A
:100C0000FDFD064605E002E1FFF7F8FD801B022826
:100C1000C0D820688007F7D52068296920F0F8003F
:100C200040EAC10020600DE0C8F80090FFF7E6FD43
:100C3000064604E0FFF7E2FD801B02281FD820686B
:100C40008007F7D42878000722D5724E7448696966
:100C50006C3671B101210160FFF7D0FD074604E059
:100C6000FFF7CCFDC01B022809D830688007F7D5F4
:100C70000EE0C0F80090FFF7C1FD074605E083E0F5
:100C8000FFF7BCFDC01B02287ED830688007F7D470
:100C90002878400768D5DFF87CA100270AF1380AD8
:100CA000DAF80000C0000BD4DAF8001041F08051EF
:100CB000CAF80010DAF80000012700F08050009018
:100CC000584E3068C00510D4306840F480703060F1
:100CD000FFF794FD009005E0FFF790FD0099401AA2
:100CE000022851D83068C005F6D54A4EA868683643
:100CF00001280FD00528306810D020F001003060A6
:100D0000306820F004003060A868B8B1FFF776FDC5
:100D100000900FE0306840F00100F4E740F004007C
:100D20003060F7E7FFF76AFD0099411A41F2883019
:100D3000814264D830688007F4D50EE0FFF75EFD8D
:100D4000009007E0FFF75AFD0099411A41F2883000
:100D5000814254D830688007F4D42FB1DAF80010FB
:100D600021F08051CAF80010A869C0B3DBF8001068
:100D7000C1F3810102294AD00228484607D0C8F8A9
:100D80006000FFF73BFD00E039E005463AE04746EA
:100D9000C8F86000FFF732FD064604E0FFF72EFDBD
:100DA000801B02282BD820688001F7D4D5E90701E1
:100DB0000843A96A1C4A490802EB01416A6A41EAF0
:100DC0008211084395F82C1040EA01611148001F78
:100DD000016001203866FFF711FD054605E014E0CB
:100DE000FFF70CFD401B022809D820688001F7D5C9
:100DF0000BE000BFFFF702FD401B022802D90320D1
:100E0000BDE8F88F20688001F4D40020F8E70120C5
:100E1000F6E7000008380240003802400000474270
:100E2000800E4742007000400000FFFF10B5401EDA
:100E3000B0F1807F01D3012010BD4FF0E02460614C
:100E40000F21601700F0B4FD0020A0610720206191
:100E5000002010BD7047000070B50268044610689D
:100E6000D168536910F00F0F50D003F0010501F461
:100E7000907635435DD0C20705D0CA0503D5E26B35
:100E800042F00102E263420705D5DA0703D0E26BC4
:100E900042F00202E263820705D5DA0703D0E26B73
:100EA00042F00402E263020705D5DA0703D0E26BE1
:100EB00042F00802E263E26B002A33D0800604D5D8
:100EC000880602D5204600F03DFB20684069E16BB2
:100ED000C0F38010090700D428B3204600F024FB9B
:100EE0002068416949061AD5416921F040014161F4
:100EF000606BA0B11B490165606BFFF7E5FA002844
:100F000010D0606B016DBDE870400847830610D5B6
:100F10008B060ED52046BDE8704000F013BB20467E
:100F2000FFF798FF70BD2046FFF794FF0020E063B5
:100F300070BD030606D50B0604D52046BDE87040FB
:100F400000F0A2BC4006F3D54806F1D5D168204692
:100F500021F04001D160202184F8391000F0D5F94A
:100F600070BD00001915010870B5040004D094F894
:100F70003900002510B106E0012070BD84F838501A
:100F8000204600F023F8242084F839002068C16846
:100F900021F40051C160204600F020FB2068016967
:100FA00021F4904101612068416921F02A014161E9
:100FB0002068C16841F40051C160E563202084F8D5
:100FC000390084F83A00002070BD0000F0B587B009
:100FD000044614216846FFF72DF93A48384E256833
:100FE00038491038022201230324B5421FD10D686D
:100FF00045F400250D60096801F4002105910168A0
:1010000041F0040101600068694600F004000590A9
:10101000A0028DE81D00082004902B48FFF710FB6C
:10102000002211463420FFF757FC342022E0274FDE
:101030000726BD4222D12349091D0D6845F0100540
:101040000D60096801F010010591016841F002018D
:1010500001600068694600F002000590C0208DE83C
:101060005D001B48FFF7ECFA002211462520FFF730
:1010700033FC2520FFF722FC07B0F0BD154FBD4221
:10108000FAD10D6845F400350D60096801F40031AE
:101090000591016841F0080101600068694600F0AF
:1010A0000800059060208DE85D000B48FFF7C8FA46
:1010B000002211462620FFF70FFC2620DAE7000069
:1010C000004C00404038024000080240001001403F
:1010D0000004024000440040000C024090F83A3006
:1010E000202B22D1F9B1F2B190F83830012B1CD06D
:1010F00081628285C2850021C163222280F83A2064
:1011000080F838100168CA6842F48072CA600168C9
:101110004A6942F001024A610068C16841F0200159
:10112000C160002070470120704702207047000016
:101130002DE9F04100683B49884242D13A4C606851
:1011400001280AD000283CD104F114052878FF2892
:1011500037D16878012836D04DE034A0A16800F07E
:1011600017FC0025344E354F2561206906EB8001C0
:1011700016F82030CA7802EB03624B7889781B049A
:1011800003EB01211144A26800EB820047F8201014
:101190002BA000F0FDFB2069401C20610428E4DB4B
:1011A000D4E90210401E814208D100F00DFE00F08B
:1011B000E9FD00F0DBFB6560E560A560A068401C10
:1011C000A060BDE8F081A8790D28FAD14FF6FF7331
:1011D000012215491C4800F03BF801206060A97805
:1011E000E87801EBC10202EB011100EB8100E06045
:1011F0002878FF28E5D16878022808D1A8790D2839
:10120000DFD112A000F0C4FB2878FF28D9D168787C
:101210000328D6D1A8790D28D3D1BDE8F0410BA081
:1012200000F0B6BB004C004000000020726F773A1F
:1012300025640D0A00000000B0380120709C0020D9
:1012400025780D0A00000000C03801206F6B0000F7
:101250002DE9F843044690F839001F4616460D461E
:10126000202850D1A5B19EB194F8380001284AD069
:10127000012084F838004FF00008C4F83C80212099
:1012800084F83900FFF7BAFAA6848146E68426E09E
:101290000120BDE8F883E08C401EE084A0684B4646
:1012A000B0F5805F4FF000024FF0800120460097BC
:1012B00003D000F01AFBE8B90DE000F016FBC8B946
:1012C00028882168C0F308004860206908B16D1CB7
:1012D00005E0AD1C03E0216815F8010B4860E08CC7
:1012E0000028D8D14B46002240212046009700F02C
:1012F000FCFA08B10320CCE7202084F8390084F8F8
:1013000038800020C5E70220C3E77047FEE70000F1
:1013100070B586B014216846FEF78CFF164800248D
:10132000016841F008010160016801F008010591C0
:10133000016841F004010160016801F004010591B8
:10134000016841F00201016000680C4E00F00200EB
:101350004FF470450590002229463046FFF748FAC1
:1013600001200095CDE90104694630460394FFF75A
:1013700067F906B070BD000030380240000C024032
:101380000C4810B50A4901604FF4E1314160002179
:1013900081600C22C160C0E904128161C161FFF764
:1013A000E3FD002803D0BDE81040FEF781BF10BD6B
:1013B000004C0040C03801200C4810B50A490160BB
:1013C0004FF4E1314160002181600C22C160C0E92D
:1013D00004128161C161FFF7C7FD002803D0BDE899
:1013E0001040FEF765BF10BD00100140003901201C
:1013F0000C4810B50A4901604FF4E1314160002109
:1014000081600C22C160C0E904128161C161FFF7F3
:10141000ABFD002803D0BDE81040FEF749BF10BD6A
:101420000044004040390120FEE770477047704794
:10143000FFF7EAB930B593B030216846FEF7FAFEFF
:1014400014210CA8FEF7F6FE18480025016841F0AB
:1014500080510160006800F08050119014480168CC
:1014600041F4804101600068022400F48040119042
:101470000120039010200490009406940820CDE9E8
:1014800007504820CDE9090403200B906846FFF778
:101490003FFB0CA90F2081E83100E002CDE90F05E8
:1014A00002210CA8FFF74AFA13B030BD40380240C1
:1014B000007000401048016841F4700101600F485D
:1014C000016841F0010101600C4A002108321160FD
:1014D00002680B4B1A400260031D0A4A1A60026838
:1014E00022F48022026005480C300160024906485F
:1014F000803908607047000088ED00E00038024045
:10150000FFFFF6FE10300024000001080148FFF73D
:10151000A3BC0000C038012010B5806B0021C1853C
:10152000C184FFF797FC10BD0168CA6822F490726D
:10153000CA6001684A6922F001024A61202180F8EC
:101540003A10704710B590F83A10222901D00220C5
:1015500010BD8168B1F5805F11D001690029016873
:101560001FD0496801F07F03816A4A1C82620B70B8
:10157000C18D491E0904090CC18518D02BE00269F0
:10158000816A002A0268526805D0D2B20A80816A54
:10159000491C8162ECE7C2F308020A80816A891C57
:1015A000F7E74A68816A4B1C83620A70E0E70168CA
:1015B000CA6822F02002CA600168CA6822F48072F8
:1015C000CA6001684A6922F001024A61202180F85C
:1015D0003A10FFF7ADFD002010BD00002DE9F041ED
:1015E000044600680169E26821F440511143016139
:1015F0002169A068E26908436169114322680843D0
:10160000D16849F20C6399430143D1602068416974
:10161000A26921F4407111434161E2696425B2F588
:10162000004F9748974922684FF032083FD08A42CE
:1016300001D082427CD1FFF729FA00EBC00101EB17
:10164000001061688900B0FBF1F6FFF71FFA00EBAC
:10165000C00101EB001061688900B0FBF1F0B0FB44
:10166000F5F06FF01801484306EB800108EB01101C
:10167000B0FBF5F000F0F006FFF708FA00EBC00150
:1016800001EB001061688900B0FBF1F0B0FBF5F0F0
:1016900006EB0016FFF7FAF900EBC00101EB0010B2
:1016A00061688900B0FBF1F7FFF7F0F9D2E08A42F8
:1016B00001D082423DD1FFF7E9F900EBC00101EB17
:1016C000001061684900B0FBF1F0B0FBF5F00601D5
:1016D000FFF7DCF900EBC00101EB00106168490085
:1016E000B0FBF1F7FFF7D2F900EBC00101EB0010FE
:1016F00061684900B0FBF1F0B0FBF5F06FF0180144
:10170000484307EB800108EBC100B0FBF5F000F0A7
:10171000F80006EB4006FFF7B9F900EBC00101EB5A
:10172000001061684900B0FBF1F7FFF7AFF93CE04A
:1017300055E0FFF79BF900EBC00101EB0010616879
:101740004900B0FBF1F0B0FBF5F00601FFF78EF9B0
:1017500000EBC00101EB001061684900B0FBF1F73C
:10176000FFF784F900EBC00101EB0010616849004C
:10177000B0FBF1F0B0FBF5F06FF01801484307EB58
:10178000800108EBC100B0FBF5F000F0F80006EBBB
:101790004006FFF76BF900EBC00101EB0010616838
:1017A0004900B0FBF1F7FFF761F900EBC00101EB75
:1017B000001061684900B0FBF1F0B0FBF5F06FF08C
:1017C0001801484307EB800108EBC100B0FBF5F0BE
:1017D00000F00700216830448860BDE8F081FFF721
:1017E00045F900EBC00101EB001061688900B0FB16
:1017F000F1F6FFF73BF900EBC00101EB0010616867
:101800008900B0FBF1F0B0FBF5F06FF01801484330
:1018100006EB800108EB0110B0FBF5F000F0F006DC
:10182000FFF724F900EBC00101EB001061688900AB
:10183000B0FBF1F0B0FBF5F006EB0016FFF716F980
:1018400000EBC00101EB001061688900B0FBF1F70B
:10185000FFF70CF900EBC00101EB00106168890093
:10186000B0FBF1F0B0FBF5F06FF01801484307EB67
:10187000800108EB0110B0FBF5F000F00F00A9E7C4
:10188000001401400010014090F83910212901D0C6
:10189000022070478168B1F5805F016A0BD04A1C55
:1018A0000262026809785160C18C491E0904090C62
:1018B000C1840ED017E009880268C1F308015160A5
:1018C00001690029016A02D0491C0162ECE7891C08
:1018D000FBE70168CA6822F08002CA600068C1683C
:1018E00041F04001C160002070472DE9F041984669
:1018F00017460E460446069D1DE0681C1BD02DB100
:10190000FEF77CFFA0EB0800A84214D92068C1684C
:1019100021F4D071C1602068416921F00101416169
:10192000202084F8390084F83A00002084F8380038
:101930000320BDE8F0812068006836EA000004D08A
:101940000020B842D9D00020F3E70120F9E70000D9
:101950000148FFF781BA0000003901200148FFF774
:101960007BBA000040390120FEE700000649086804
:10197000064A1040B0F1005F04D14868096881F35D
:101980000888004770470000000001080000FE2F93
:101990000FB4054B10B503A9044A029800F028F8CB
:1019A00010BC5DF814FB0000B11C01082C000020E5
:1019B0000907090E002804DB00F1E02080F800147C
:1019C000704700F00F0000F1E02080F8141D704710
:1019D00002E008C8121F08C1002AFAD170477047F8
:1019E000002001E001C1121F002AFBD17047000056
:1019F0002DE9FF4F8DB09B460F460446002606E0BA
:101A000025280BD05A460F999047641C761C2078E5
:101A10000028F5D111B03046BDE8F08F0025A8466A
:101A20000122984900E0054314F8013F203B02FAE7
:101A300003F00842F7D120782E2817D114F8010FAF
:101A400045F004052A280ED06FF02F022078A0F16F
:101A5000300109290AD808EB880102EB410100EBAB
:101A60000108641CF2E757F8048B641C20786C288A
:101A70000DD004DC4C2812D06A2811D104E074285F
:101A80000DD07A280CD10AE045F4001507E0617802
:101A900045F48015814202D1641C05F58015641C53
:101AA0002078692844D008DC0028B3D0582867D0B3
:101AB00063280FD0642808D13AE0702865D07328D5
:101AC00012D075285AD078285AD05A460F99904784
:101AD000761CD5E017F8040B8DF8000000208DF877
:101AE0000100E946012003E057F8049B4FF0FF3066
:101AF00069074FF0000501D40AE06D1C45450DDA79
:101B00008542FADB19F805100029F6D106E06D1CB4
:101B10008542FCDB19F805100029F8D12E4404E0B9
:101B200019F8010B5A460F9990476D1EF8D2A7E09D
:101B30000A200021CDE90801C5F3025002280CD08B
:101B400001CFC117021E71F100020CDA0023D0EBA5
:101B5000030063EB01012D2208E0FF1D27F00707BA
:101B6000F7E80201EEE72A0504D52B228DF828209C
:101B700001223CE0EA073AD02022F7E70A2000E001
:101B800010200021CDE9080107E01020002145F0D8
:101B90000405CDE908014FF00808C5F302500228FA
:101BA00010D001CF00214FF0000A2A0720D522785B
:101BB000702A0DD0DDE908C38CF0100C5CEA030C30
:101BC0000CD015E0FF1D27F00707F7E80201EAE750
:101BD00040228DF828204FF0010A0CE050EA010362
:101BE00006D030238DF828308DF829200222924625
:101BF0002278582A04D024A20DF120090B9209E082
:101C000026A2F9E7DDE90823FEF7DCFA0B9B9B5CD3
:101C100009F8013D50EA0102F4D1ADEB0900203092
:101C20000890680701D44FF001080899884503DD42
:101C30000898A8EB000000E000208046002506E0A0
:101C40000AA85A46405D0F9990476D1C761C554571
:101C5000F6DB04E030205A460F999047761CB8F125
:101C60000001A8F10108F5DC05E019F8010B5A465E
:101C70000F999047761C0899481E08900029F4DCBB
:101C8000641CC4E60928010030313233343536375C
:101C900038396162636465660000000030313233B8
:101CA0003435363738394142434445460000000058
:101CB00001B54FF6FF73012269460248FFF7C8FAE3
:101CC000009808BDC0380120FEF7A6FDFFF7B2FB63
:101CD000FFF71EFBFFF78CFBFFF752FBFFF76CFBD8
:101CE0000AA0FFF755FE17A0FFF752FE07A0FFF767
:101CF0004FFE214C606828B1204910222048FFF790
:101D0000EDF9F7E71C4907221431F7E70A2D2D2DCD
:101D10002D2D2D2D2D2D2D2D2D2D2D2D2D2D2D2DF3
:101D20002D2D2D2D2D2D2D2D2D2D2D2D2D2D2D2DE3
:101D30002D2D2D2D2D2D2D2D2D2D2D2D2D2D2D0AF6
:101D4000000000000A202020202020202020202029
:101D500020202020202053544D3332463420494146
:101D600050204150503220202020202020202020B0
:101D70002020202020200A0000000020B038012070
:101D8000C038012070B50B4C00200B4E0B4D20616C
:101D90000AE000BF56F8201045F8201008A0FFF711
:101DA000F7FD2069401C2061E168B0EB810FF1DB99
:101DB00070BD00000000002000000108300000207D
:101DC00025780D0A0000000070B588B0FEF722FCEF
:101DD0000220049004200290002501200390009529
:101DE00006A906956846FEF781FB0D4C0E4E25614F
:101DF0000C4D20690BE000BF55F8202006EB800158
:101E000000230220FEF7C8FB2069401C2061E16826
:101E1000B0EB810FF0DBFEF7B5FB08B070BD000042
:101E200000000020709C002000000108000000005D
:101E3000000000000102030406070809000000007A
:101E400001020304641E01080000002030000000AD
:101E5000D0190108941E010830000020707901009B
:101E6000E0190108790000000000000000000000F7
:101E70000000000000000000FFFF000000000D0057
:101E80000100000010000000000000000024F40029
:041E9000000000004E
:040000050801018964
:00000001FF
